:100000003AC0000053C0000051C00000D8C1000039
:100010004DC000004BC0000049C0000047C00000B8
:1000200045C0000043C0000041C0000000C2000005
:100030003DC000003BC0000039C0000037C00000D8
:1000400035C0000033C0000031C000002FC00000E8
:100050002DC000002BC0000029C0000027C00000F8
:1000600025C0000023C00000760184019201A00198
:10007000AE01BC01CA0111241FBECFEFD4E0DEBF28
:10008000CDBF11E0A0E0B1E0E2E0F9E002C00590F0
:100090000D92A431B107D9F721E0A4E1B1E001C08C
:1000A0001D92A83AB207E1F7BBD029C4A9CF43E01B
:1000B00050E091E0282F30E0092E02C035952795B9
:1000C0000A94E2F78227990F4150510999F7089550
:1000D00010921C0183B1877080930A0190910901ED
:1000E00080910A01981709F455C080910A01809304
:1000F000090180919B0190919C0180FF06C0809135
:100100000A018095877080930A0180919B019091EC
:100110009C0181FF05C080910A01C9DF80930A011B
:1001200020919B0130919C0190910A012227307708
:10013000832F82958F70890F877080930A01809139
:100140000A0190E0880F991F0796D4D39093A701D6
:100150008093A6018091A6019091A701C3D38093BB
:100160001401409114016091A6017091A70150E023
:100170006F5F7F4F80E291E0A5D380E197E290939B
:1001800008018093070183B5816083BD10928500CB
:10019000109284008091A1019091A201892BC9F055
:1001A00020910701309108018091A1019091A20155
:1001B0002817390774F0109208011092070181E0A6
:1001C00080931C0110929E0110929D0110921D01BE
:1001D0001EC08091200190E090939E0180939D012C
:1001E00089B1887390E095958795959587959595B4
:1001F000879580931D0180919B0190919C0180FFC8
:1002000006C080911D018095877080931D01E0914B
:100210001D01F0E0E55FFE4F80818093A30108950A
:1002200080E090E05FD38430F1F781E090E062D32A
:1002300090939C0180939B0180919B0190919C01E4
:10024000807F9927929582958F7089279F70892743
:1002500048E552E0849F9001859F300D949F300DBA
:1002600011243093A2012093A10183E090E042D3B6
:100270009093A5018093A40187E085B980E284B9B9
:100280008CE38BB980E48AB9E0E8F0E08081806893
:100290008083EFE6F0E080818260808382E085BD2C
:1002A000E0E0F0E089E08093570084918F70823025
:1002B00071F4E1E8F0E080818D6080838DE487BD9A
:1002C00081E690E0909389008093880075C0E0916A
:1002D0009B01F0919C01EF2FFF27E770FF27E7308C
:1002E000F10508F064C0EC5CFF4FE6C28FE487BD07
:1002F000E1E8F0E080818B6080838FEF91E3909361
:1003000089008093880053C083EB87BDE1E8F0E06B
:1003100080818B6080838FE790E790938900809342
:10032000880045C08CE787BDE1E8F0E080818B6004
:1003300080838FE19EE4909389008093880037C08A
:1003400081E687BDE1E8F0E080818B60808388E012
:100350009DE3909389008093880029C08DE487BD38
:10036000E1E8F0E080818B60808383ED90E39093FF
:100370008900809388001BC08CE987BDE1E8F0E02C
:1003800080818B60808387EA91E6909389008093D7
:1003900088000DC087E987BDE1E8F0E080818B60CF
:1003A000808386E39FE5909389008093880084E0B2
:1003B0008093680080936D008BDE7894FFCF1F924E
:1003C0000F920FB60F9211248F939F934A9B28C0D0
:1003D0008091010190910201019790930201809315
:1003E0000101892BE9F480911E0190911F019093E6
:1003F00002018093010180911901882389F081E035
:1004000090E090930401809303018093180110926F
:10041000190183B5816083BD10928500109284001C
:100420009F918F910F900FBE0F901F9018951F9264
:100430000F920FB60F9211242F933F934F935F9318
:100440006F937F938F939F93AF93BF93CF93DF93DC
:10045000EF93FF93809117019FEF980F90931701EF
:10046000811117C2809116018093170180910701B5
:100470009091080101969093080180930701809163
:10048000030190910401019790930401809303016B
:10049000892B29F080911801882391F0FAC180916D
:1004A000A4019091A5019093040180930301809190
:1004B0001801882319F081E08093A301109218019C
:1004C00080911A0190911B01892B79F080911A017A
:1004D00090911B01019790931B0180931A01892B26
:1004E00009F0D7C181E08093A3018091A3018150DD
:1004F0008093A3018111CDC1E0911D01F0E0E55F82
:10050000FE4F80818093A301809115018938E1F02D
:10051000809115018838C1F0809115018039A1F0D2
:10052000809115018F3881F0809115018A3861F032
:10053000809115018B3841F080911501893B21F0A4
:10054000809115018A3B49F486EF809306018FEF75
:10055000809305018FEE8093000180910601815008
:100560008093060188230CF079C1809105018823CE
:1005700034F08091050188230CF49FC0A1C08091C4
:1005800015018F3E29F4809106018A3F0CF081C14C
:10059000809106018E3F6CF37CC19ADD809114013D
:1005A00020919D0130919E0190E002978217930760
:1005B000A4F380919D0190919E019C012F5F3F4F7C
:1005C00030939E0120939D01FC01E05EFE4F8181EE
:1005D0008093150180911501887F803899F480916E
:1005E0001C0181110DC080911501877080931D0140
:1005F000E0911D01F0E0E55FFE4F80818093A30153
:100600001092150180911501882341F28091150106
:100610008D3859F480919B0190919C018C709927A1
:10062000089709F42E98D0931501809115018E3802
:1006300059F480919B0190919C018C7099270897A7
:1006400009F42E9AD093150180919B0190919C0101
:100650008C709927049739F480911D01882311F03B
:100660002E9801C02E9AC09305018091150120910A
:10067000050190E002C0959587952A95E2F780FFE5
:1006800011C0809105018150809305018091150171
:100690002091050190E002C0959587952A95E2F793
:1006A00080FDEFCF809105018150809305018091FD
:1006B000050188230CF472CF03C0DBEBC7E06ECFDB
:1006C00080911C01882339F0809115018A3819F432
:1006D0008FEE80931501809115018B3809F495C038
:1006E00070F4883809F44BC020F48C3709F47DC0CD
:1006F00099C0893801F18A3809F481C093C08039E2
:1007000009F460C020F48F3809F466C08BC08B3BBD
:1007100009F481C08F3E09F085C0809100018F3EB1
:1007200019F41092060103C08DEF809306018FEF3C
:10073000809305018FC081E08093060180919D0127
:1007400090919E019C012F5F3F4F30939E0120931B
:100750009D01FC01E05EFE4F818190E09C01220F33
:10076000331F880F991F880F991F880F991F820FB9
:10077000931F019790931B0180931A016BC01092F5
:10078000060180919D0190919E019C012F5F3F4F3A
:1007900030939E0120939D01FC01E05EFE4F81811C
:1007A00090E09C01220F331F880F991F880F991F1B
:1007B000880F991F820F931F019790931B018093BD
:1007C0001A0148C081E08093060189E090E090938F
:1007D0001B0180931A013EC01092060189E090E04F
:1007E00090931B0180931A0135C083B7817F846089
:1007F00083BFF89483B7816083BF88952BC081E065
:10080000809318011092060125C081E080931801A1
:10081000809306011FC086EF809306018FEF8093BF
:10082000050118C0809115012091050190E002C0DA
:10083000959587952A95E2F780FF04C083E0809321
:10084000060103C081E0809306018091050181507B
:10085000809305018091150180930001809106012C
:10086000181664F42D9A80919B0190919C018C70D4
:100870009927892B71F482E484BD0BC02D98809157
:100880009B0190919C018C709927892B11F482E037
:1008900084BDFF91EF91DF91CF91BF91AF919F9177
:1008A0008F917F916F915F914F913F912F910F9019
:1008B0000FBE0F901F901895EE0FFF1F0590F4913B
:1008C000E02D0994DC01CB01FC01F999FECF06C0B3
:1008D000F2BDE1BDF89A319600B40D9241505040FE
:1008E000B8F70895F999FECF92BD81BDF89A99277E
:1008F00080B50895A8E1B0E042E050E0E5CFF8947B
:02090000FFCF27
:10090200EF01000100FFF61027626301020A1E3C9C
:0409120064962C00BB
:00000001FF
